:1000000012C02BC02AC029C028C027C026C025C0C6
:1000100024C023C022C021C020C01FC01EC01DC0DC
:100020001CC01BC01AC011241FBECFE5D4E0DEBF28
:10003000CDBF10E0A0E6B0E0E2E0F1E002C0059044
:100040000D92A036B107D9F710E0A0E6B0E001C0EC
:100050001D92A036B107E1F72CC0D2CF40E050E0AE
:100060004817590768F420E030E0275E3F4F60E70B
:100070002E343607D0F34F5F5F4F4817590798F378
:10008000089580B7846080BF87B38F6387BB88B3D0
:10009000817E816288BB84B3837C836084BB85B3AB
:1000A000807C85BB81B384EF81BB82B380E282BB5D
:1000B0000895CFE5D4E0DEBFCDBF85B5887F85BD8F
:1000C000E0DF82B38F7E806282BB88B3806388BBAF
:1000D000C19A87E090E0C2DFC1988F9A979AA19861
:1000E000A99881E090E0BADF999B03C0A19AA99AF0
:1000F00002C0A19AA9988F9A979884E690E0AEDF03
:02010000E7CF47
:00000001FF
